:1000000023C03BC03AC039C0E5C037C036C035C098
:1000100034C033C032C02FC12EC139C138C143C131
:1000200042C12DC12CC137C136C141C140C10BC134
:1000300099C1A2C1AEC1B7C1C3C1CCC1D8C1E1C1D0
:10004000EDC1F6C102C20BC211241FBECFEDCDBF60
:1000500010E0A0E6B0E0E4E1F5E003C0C895319619
:100060000D92A036B107D1F710E0A0E6B0E001C0D4
:100070001D92AE36B107E1F72CC2C2CFF92FE82F9F
:1000800080818F5F80838C3389F5108281818F5FBF
:1000900081838C3359F5118282818F5F828388310D
:1000A00029F5128283818F5F8383803211F08F3133
:1000B00011F4848105C08E3129F48481823071F479
:1000C0008F5F09C08D3151F48481823039F485818C
:1000D000837021F083E0848381E0838384818D3089
:1000E00029F481E0848385818F5F85830895089555
:1000F000F92FE82F32814AE0832F642FFFD1282F78
:100100002295207F832FFAD1292B88B3887F88BB43
:10011000C29A22BB0895F92FE82F31814AE0832F3C
:10012000642FECD1282F2295207F832FE7D1292B14
:1001300088B3887F88BBC19A22BB0895F92FE82F26
:1001400030814AE0832F642FD9D1282F2295207F38
:10015000832FD4D1292B88B3887F88BBC09A22BB38
:100160000895F92FE82F33814AE0832F642FC6D1F9
:10017000282F2295207F832FC1D1292B88B3887FF8
:1001800088BBC29A22BB0895F92FE82F34814AE038
:10019000832F642FB3D1282F2295207F832FAED1B8
:1001A000292B88B3887F88BBC19A22BB0895F92F79
:1001B000E82F35814AE0832F642FA0D1282F229584
:1001C000207F832F9BD1292B88B3887F88BBC09A3F
:1001D00022BB08951F920F920FB60F9211242F93F6
:1001E0003F934F935F936F937F938F939F93AF93BF
:1001F000BF93EF93FF9385E998E99BBD8ABD8091FA
:100200006100815080936100882359F480916D00D2
:10021000813019F082E690E031DF85E199E99BBDFC
:100220008ABD80916D00813099F480916B0099278F
:10023000AA27BB27F92FE82F3197ED30F105D0F52C
:10024000E55FFF4F099410926D0010926B0032C071
:1002500080916A00992781309105A9F0823091053B
:100260001CF4892B21F026C00297C9F023C080918D
:100270006800882321F082E690E03ADF1BC082E626
:1002800090E06FDF17C080916800882321F082E63C
:1002900090E041DF0FC082E690E076DF0BC08091F6
:1002A0006800882321F082E690E048DF03C082E600
:1002B00090E07DDF80916A008F5F80936A008330D9
:1002C00011F410926A00B39906C080916C008F5FA0
:1002D00080936C0005C010926C0081E080936900EF
:1002E000B49906C0809160008F5F8093600005C064
:1002F0001092600081E08093690080916C008931E8
:10030000A1F480916D00882351F0809169008823C9
:1003100031F080916B008F5F80936B000FC08091F4
:10032000680080958093680009C0883C39F481E0BA
:1003300080936D0080936B00109269008091600043
:10034000893109F098C080916B009927AA27BB27B3
:10035000F92FE82F3197EC30F10508F08CC0E85EFA
:10036000FF4F099480916400843110F0845101C0E2
:10037000865F809364007FC020916400822F6AE0D2
:10038000BDD0993011F4295001C02F5F2093640033
:1003900072C080916300823310F0825301C0865F87
:1003A0008093630068C020916300822F6AE0A6D02A
:1003B000993011F4295001C02F5F209363005BC076
:1003C00080916200823310F0825301C0865F809377
:1003D000620051C020916200822F6AE08FD0993074
:1003E00011F4295001C02F5F2093620044C0809116
:1003F00065008E3110F08E5101C0865F80936500DC
:100400003AC020916500822F6AE078D0993011F4CB
:10041000295001C02F5F209365002DC08091660098
:100420008A3010F08A5001C0865F8093660023C036
:1004300020916600822F6AE061D0993011F4295032
:1004400001C02F5F2093660016C08091670086343C
:1004500010F0865401C0865F809367000CC0209125
:100460006700822F6AE04AD0993011F4295001C008
:100470002F5F20936700FF91EF91BF91AF919F9104
:100480008F917F916F915F914F913F912F910F903D
:100490000FBE0F901F9018952FEF21BB87E087BBF1
:1004A00028BB89E08EBD85E998E99BBD8ABD1DBC4E
:1004B0001CBC1092610080E489BF209368001092F8
:1004C0006D0010926C001092600010926A00789497
:1004D0000895CFEDD0E0DEBFCDBF95E090936700EB
:1004E00081E08093660080936500909364008AE0C9
:1004F0008093630090936200CFDFFFCF991B79E078
:1005000004C0991F961708F0961B881F7A95C9F7A3
:040510008095089535
:00000001FF
